:1000000019C033C032C031C030C02FC02EC02DC087
:100010002CC02BC02AC029C0CCC027C026C025C0F8
:1000200024C023C022C021C020C01FC01EC01DC0CC
:100030001CC01BC011241FBECFEFD2E0DEBFCDBF5E
:1000400011E0A0E0B1E0ECE9F9E002C005900D920A
:10005000AA30B107D9F711E0AAE0B1E001C01D92C2
:10006000A436B107E1F7C0D197C4CACF80648093AA
:100070007C0080917A00806480937A0080917A007D
:1000800086FDFCCF2091780030917900C901089558
:10009000CF93DF9380914301803110F010924301A0
:1000A00080914301C82FD0E0CC0FDD1FC65EDE4F2C
:1000B0002881398140E050E080911601909117012C
:1000C000A0911801B0911901821B930BA40BB50BE1
:1000D0008093160190931701A0931801B093190112
:1000E00082E0C4DF9983888380914301C82FD0E0E8
:1000F000CC0FDD1FFE01E65EFE4F2081318140E026
:1001000050E08091160190911701A0911801B091D3
:100110001901820F931FA41FB51F8093160190939E
:100120001701A0931801B0931901CC5BDE4F288111
:10013000398140E050E08091120190911301A0912B
:100140001401B0911501821B930BA40BB50B809386
:10015000120190931301A0931401B093150183E051
:1001600085DF9983888320914301E22FF0E0EE0F31
:10017000FF1FEC5BFE4F4081518160E070E0809199
:10018000120190911301A0911401B0911501840FF7
:10019000951FA61FB71F8093120190931301A09380
:1001A0001401B09315012F5F20934301DF91CF918C
:1001B00008951F920F920FB60F9211242F933F9321
:1001C0004F935F936F937F938F939F93AF93BF935F
:1001D00080910801882309F463C080910A019091FD
:1001E0000B01A0910C01B0910D01803020E092072D
:1001F00021E0A20720E0B20718F49C01AD0113C072
:100200008F3F2FEF920721E0A20720E0B20728F0EE
:100210002FEF3FEF40E050E006C09C01AD01569546
:10022000479537952795821B930BA40BB50B8093AD
:100230000A0190930B01A0930C01B0930D01609102
:100240008A0070918B00620F731F70938B00609314
:100250008A000097A105B10509F09EC080E2809355
:1002600080008091040190910501A0910601B09158
:10027000070120910001309101014091020150914C
:100280000301821B930BA40BB50B80930E0190937B
:100290000F01A0931001B0931101109208017CC0CE
:1002A00080910E0190910F01A0911001B091110168
:1002B000803020E0920721E0A20720E0B20718F486
:1002C0009C01AD0113C08F3F2FEF920721E0A207E1
:1002D00020E0B20728F02FEF3FEF40E050E006C0EB
:1002E0009C01AD015695479537952795821B930B39
:1002F000A40BB50B80930E0190930F01A0931001F6
:10030000B093110160918A0070918B00620F731F8E
:1003100070938B0060938A000097A105B105E1F509
:1003200081E08093080180E3809380008091000148
:1003300090910101A0910201B091030180930A0103
:1003400090930B01A0930C01B0930D0180913E019D
:10035000882311F180913F0190914001A0914101CA
:10036000B09142018093040190930501A09306018E
:10037000B093070180913A0190913B01A0913C011B
:10038000B0913D018093000190930101A09302017F
:10039000B093030110923E01BF91AF919F918F9155
:1003A0007F916F915F914F913F912F910F900FBE71
:1003B0000F901F901895E1E8F0E0108210928500F0
:1003C0001092840081E0808310928B0010928A004A
:1003D00084E086BBEFE6F0E080818460808387E87C
:1003E00080937A0078940895DF92EF92FF920F93B2
:1003F0001F9380E8809361001092610084E084B9CB
:1004000082E085B9D8DFDD24D39442DE80913E01BD
:100410008823D9F7199BF9CF6091160170911701C4
:100420008091180190911901A2D120E030E040E8BC
:100430005DE34FD220E030EC4FE754E404D120E0FC
:1004400030E44CE156E445D27B018C017F2D912FA5
:1004500020E030E040E251E4F2D0882324F4EE249E
:10046000FF2400E211E460E876E988E19BE42E2DA8
:100470003F2D402F512FE7D020E030E040E05FE3F8
:100480007AD049D160933F0170934001809341013C
:1004900090934201609112017091130180911401B7
:1004A0009091150164D120E030E040E85DE311D285
:1004B00020E030EC4FE754E4C6D02DEC3CEC4CECA3
:1004C0005DE307D27B018C017F2D912F2CEA35EC67
:1004D00047E257E3B4D0882334F4FCEAEF2EE5EC8E
:1004E000FE2E07E217E36E2D7F2D802F912F20E83F
:1004F00036E948E15BE4EDD120E030E040E05FE345
:100500003AD009D160933A0170933B0180933C014A
:1005100090933D0120913A0130913B0140913C0183
:1005200050913D0180913F0190914001A091410186
:10053000B0914201845F9140A040B0408217930780
:10054000A407B507A0F480913F0190914001A091CC
:100550004101B0914201845F9140A040B04080933E
:100560003A0190933B01A0933C01B0933D01D0929E
:100570003E014BCF5058BB27AA270ED070C161D186
:1005800030F066D120F031F49F3F11F41EF456C1D3
:100590000EF4E095E7FB4CC1E92F72D180F3BA1756
:1005A000620773078407950718F071F49EF58AC1F6
:1005B0000EF4E0950B2EBA2FA02D0B01B90190017E
:1005C0000C01CA01A0011124FF27591B99F0593FC2
:1005D00050F4503E68F11A16F040A22F232F342F0A
:1005E0004427585FF3CF469537952795A795F04058
:1005F0005395C9F77EF41F16BA0B620B730B840B6D
:10060000BAF09150A1F0FF0FBB1F661F771F881F24
:10061000C2F70EC0BA0F621F731F841F48F487957C
:1006200077956795B795F7959E3F08F0B3CF93956B
:10063000880F08F09927EE0F979587950895D4D0E5
:1006400008F481E008950CD00AC102D140F0F9D03D
:1006500030F021F45F3F19F0EBC0511134C1EEC00E
:100660000FD198F39923C9F35523B1F3951B550B7B
:10067000BB27AA2762177307840738F09F5F5F4F75
:10068000220F331F441FAA1FA9F333D00E2E3AF0B6
:10069000E0E830D091505040E695001CCAF729D0D0
:1006A000FE2F27D0660F771F881FBB1F261737071F
:1006B0004807AB07B0E809F0BB0B802DBF01FF274F
:1006C00093585F4F2AF09E3F510568F0B1C0FBC0C0
:1006D0005F3FECF3983EDCF3869577956795B79589
:1006E000F7959F5FC9F7880F911D9695879597F9A4
:1006F0000895E1E0660F771F881FBB1F621773071D
:100700008407BA0720F0621B730B840BBA0BEE1F31
:1007100088F7E0950895BCD088F09F5790F0B92FE6
:100720009927B751A0F0D1F0660F771F881F991F46
:100730001AF0BA95C9F712C0B13081F0C3D0B1E058
:100740000895C0C0672F782F8827B85F39F0B93F68
:10075000CCF3869577956795B395D9F73EF4909548
:100760008095709561957F4F8F4F9F4F0895E894C6
:1007700009C097FB3EF490958095709561957F4FE9
:100780008F4F9F4F9923A9F0F92F96E9BB27939597
:10079000F695879577956795B795F111F8CFFAF4A7
:1007A000BB0F11F460FF1BC06F5F7F4F8F4F9F4FD8
:1007B00016C0882311F096E911C0772321F09EE836
:1007C000872F762F05C0662371F096E8862F70E09C
:1007D00060E02AF09A95660F771F881FDAF7880F76
:1007E0009695879597F90895990F0008550FAA0BCC
:1007F000E0E8FEEF16161706E807F907C0F0121634
:100800001306E407F50798F0621B730B840B950B36
:1008100039F40A2661F0232B242B252B21F408958B
:100820000A2609F4A140A6958FEF811D811D089528
:1008300097F99F6780E870E060E008959FEF80EC93
:10084000089500240A941616170618060906089536
:1008500000240A9412161306140605060895092E9C
:100860000394000C11F4882352F0BB0F40F4BF2B0B
:1008700011F460FF04C06F5F7F4F8F4F9F4F08954B
:1008800057FD9058440F551F59F05F3F71F0479541
:10089000880F97FB991F61F09F3F79F08795089526
:1008A000121613061406551FF2CF4695F1DF08C045
:1008B000161617061806991FF1CF86957105610562
:1008C00008940895E894BB2766277727CB0197F90A
:1008D00008950BD0C4CFB5DF28F0BADF18F0952308
:1008E00009F0A6CFABCF1124EECFCADFA0F3959FBE
:1008F000D1F3950F50E0551F629FF001729FBB2707
:10090000F00DB11D639FAA27F00DB11DAA1F649FB2
:100910006627B00DA11D661F829F2227B00DA11D65
:10092000621F739FB00DA11D621F839FA00D611DEB
:10093000221F749F3327A00D611D231F849F600D0C
:10094000211D822F762F6A2F11249F5750408AF045
:10095000E1F088234AF0EE0FFF1FBB1F661F771FD1
:10096000881F91505040A9F79E3F510570F060CF0D
:10097000AACF5F3FECF3983EDCF3869577956795B9
:10098000B795F795E7959F5FC1F7FE2B880F911DEF
:0C0990009695879597F90895F894FFCF8D
:0A099C00A0860100400D03000100D9
:00000001FF
